:100000008A0115284B29542982073F3406345B3472
:100010004F3466346D347D3407347F346F34773435
:100020007C3439345E34793471348312860185012D
:10003000831686018312AC01AE01B001FF30831636
:10004000850080309F008312A0014130A1002E085E
:10005000A200A20DA20D220DF83921070318A00A53
:100060009F003C30AB0002208A110A1283121F1538
:1000700083121F1938281F101E08A001A90020088C
:10008000AA002908A1002A08A000A10DA00DA10D19
:10009000A00DA10DA00DA10DA00DA10DA00DA10DF4
:1000A000A00DA10DA00DA10DA00D21080039A101E9
:1000B00083161E078312A1000318A00A2108A900B5
:1000C0002008AA00AD0183122C082D02013003186C
:1000D0000301003C031995282A08A0002908A10063
:1000E000A2010A30A3001030A400A501A6018312CA
:1000F000200DA60DA50D2308A6022208031C220F21
:10010000A50203188A282308A60722080318220F2D
:10011000A50703108312A10DA00DA40B77282108B9
:10012000A9002008AA00AD0A632883122A08A000AB
:100130002908A100A2010A30A3001030A400A501E3
:10014000A6018312200DA60DA50D2308A6022208E4
:10015000031C220FA5020318B4282308A6072208AF
:100160000318220FA50703108312A10DA00DA40BE5
:10017000A1282508A0002608AF002F088600A001AE
:100180002C08043E0318A00AA000003C031DCA2846
:100190000614FA2883122008013C031DD128861476
:1001A000FA2883122008023C031DD8280615FA28D5
:1001B00083122008033C031DDF288615FA288312CA
:1001C0002008043C031DE6280616FA28831220089E
:1001D000053C031DED288616FA2883122008063CEC
:1001E000031DF4280617FA2883122008073C031D74
:1001F000FA288617033083122C02013003180301FA
:10020000003C03190529AC0A07298312AC0105300B
:100210008312A70003208A110A12FF30831685007B
:1002200006309F00831205081039003C03191B2972
:100230000130B0004A298312300803194829A0016F
:100240002E08013E0318A00AA100A2010430A30059
:100250001030A400A501A6018312200DA60DA50D46
:100260002308A6022208031C220FA50203183F2917
:100270002308A60722080318220FA50703108312DC
:10028000A10DA00DA40B2C292508A0002608AE0066
:100290008312B0011E28AB0C7F30AB050430AB02DB
:1002A000AB0B50290000080073308312A800000037
:1002B000000000000000000000000000000000003E
:1002C00000000000A80B58290000A70B54290000CB
:0202D000080024
:00000001FF
